:020000040000FA
:040000001FEF00F0FE
:08000800006ED8CF02F0E0CF3A
:1000100001F0F2B28CEC02F0F2B48CEC01F09EB084
:10002000C6EC01F09EB206EC02F0A1B243EC02F085
:1000300000D001C0E0FF005002C0D8FF1000806A6D
:10004000816A826A070EC16E000E926E946E030E74
:10005000936E80848282828C818A430ED56EF29464
:10006000F28AB40ECD6E9E909D80020ECA6E9E9254
:100070009D82F00EB16EA192A08283EC02F0CD8041
:10008000D09EF28EF28C000000000000FCD7D59EBE
:100090000B1CF6EC02F0236E0B50F6EC02F0246E13
:1000A000241CD8A468EF00F02350D8A460EF00F01F
:1000B000010E176E010E186EFF0E196E89EF00F01B
:1000C000010E176E2350186EFF08196E89EF00F0AD
:1000D000231CD8B477EF00F02350176E2450196E0C
:1000E00024042324186E175E195E89EF00F0245053
:1000F000D8B483EF00F02450186EFF08176E010E7D
:10010000196E89EF00F0FF0E176E010E186E010ECA
:10011000196E000E136E171CD66E80928090809818
:1001200080960FA080820FB08080D58E1200CD9077
:100130000C1CF6EC02F0256E0C50F6EC02F0266E6C
:10014000261CD8A4B8EF00F02550D8A4B0EF00F0DA
:10015000010E1A6E010E1B6EFF0E1C6ED9EF00F021
:10016000010E1A6E25501B6EFF081C6ED9EF00F0B1
:10017000251CD8B4C7EF00F025501A6E26501C6E0F
:10018000260425241B6E1A5E1C5ED9EF00F0265053
:10019000D8B4D3EF00F026501B6EFF081A6E010E84
:1001A0001C6ED9EF00F0FF0E1A6E010E1B6E010ED1
:1001B0001C6E000E146EFF0ECF6E1A1CCE6E829057
:1001C000809A8296829410A0828010B0808ACD801E
:1001D0001200CA940D1CF6EC02F0276E0D50F6ECDE
:1001E00002F0286E281CD8A40AEF01F02750D8A4EA
:1001F00002EF01F0010E1D6E010E1E6EFF0E1F6E4E
:100200002BEF01F0010E1D6E27501E6EFF081F6EB2
:100210002BEF01F0271CD8B419EF01F027501D6E09
:1002200028501F6E280427241E6E1D5E1F5E2BEFB4
:1002300001F02850D8B425EF01F028501E6EFF08B9
:100240001D6E010E1F6E2BEF01F0FF0E1D6E010ED5
:100250001E6E010E1F6E000E156ECC6A1D50CB6E09
:10026000829A82988194829E11A0828A11B082889B
:10027000CA841200B1900E1CF6EC02F0296E0E50EA
:10028000F6EC02F02A6E2A1CD8A45BEF01F029508C
:10029000D8A453EF01F0010E206E010E216EFF0E67
:1002A000226E7CEF01F0010E206E2950216EFF08B6
:1002B000226E7CEF01F0291CD8B46AEF01F02950BE
:1002C000206E2A50226E2A042924216E205E225E8E
:1002D0007CEF01F02A50D8B476EF01F02A50216E5D
:1002E000FF08206E010E226E7CEF01F0FF0E206EE3
:1002F000010E216E010E226E000E166EFF0EB36E01
:10030000201CB26E81988196819C819E12A081886A
:1003100012B08186B1801200D59EF294F28A030E4B
:10032000FA6E020E1302F350F92602D013D020D039
:10033000181CD66E010E136E809280908098809665
:100340000FA080820FB080800FA280880FB28086BD
:10035000D58E1200191CD66E020E136E80928090FC
:10036000809880960FA280880FB28086D58E12006A
:10037000171CD66E000E136E809280908098809627
:100380000FA080820FB08080D58E1200CD909E90FD
:100390009D80030EFA6E020E1402F350F92602D06D
:1003A00015D024D0FF0ECF6E1B1CCE6E010E146E26
:1003B0008290809A8296829410A0828010B0808A67
:1003C00010A2828610B28284CD801200FF0ECF6E02
:1003D0001C1CCE6E020E146E8290809A82968294BD
:1003E00010A2828610B28284CD801200FF0ECF6EE2
:1003F0001A1CCE6E000E146E8290809A82968294A1
:1004000010A0828010B0808ACD801200CA949E9283
:100410009D82040EFA6E020E1502F350F92602D0E8
:1004200014D022D0CC6A1E50CB6E010E156E829A6B
:1004300082988194829E11A0828A11B0828811A232
:10044000818411B2828ECA841200CC6A1F50CB6E96
:10045000020E156E829A82988194829E11A28184E6
:1004600011B2828ECA841200CC6A1D50CB6E000E6F
:10047000156E829A82988194829E11A0828A11B010
:100480008288CA841200B190A192A082040EFA6EF2
:10049000020E1602F350F92602D015D024D0FF0E1A
:1004A000B36E211CB26E010E166E81988196819CEE
:1004B000819E12A0818812B0818612A2818C12B214
:1004C000818EB1801200FF0EB36E221CB26E020E3E
:1004D000166E81988196819C819E12A2818C12B2A7
:1004E000818EB1801200FF0EB36E201CB26E000E22
:1004F000166E81988196819C819E12A0818812B08F
:100500008186B180120093809382F18CF292F288FE
:10051000036A080E046E120091EC02F0F292F28867
:100520001200D89081B2D88008320350096ED8905A
:100530000936050ED8B0E828FA6E440E0924D8B062
:10054000FA2AF96E02D00AD016D0042E1200010E3B
:10055000036E060E046E0850056E1200042E120083
:10056000020E036E080E046E0850066ED890063216
:10057000D89006321200042E1200000E036E080EF0
:10058000046E800E056212000850076E0650030BC1
:10059000086E06503C0B066E0642064200EE0FF057
:1005A000065008C0EBFF00EE0BF0065007C0EBFF53
:1005B000050EFA6E060E0602F350F92647EC00F01F
:1005C000120097EC00F01200E9EC00F012003AEC97
:0405D00001F0120024
:0405EC002B6E060E5E
:1005F000FA6E020E2B02F450FA26F350000FF96E39
:10060000000C020C030C050C060C080C090C0B0C5E
:100610000D0C0E0C100C110C130C140C160C180CE9
:10062000190C1B0C1C0C1E0C1F0C210C220C240C76
:10063000260C270C290C2A0C2C0C2D0C2F0C300C02
:10064000320C330C350C370C380C3A0C3B0C3D0C8F
:100650003E0C400C410C430C440C460C470C490C1E
:100660004A0C4C0C4D0C4F0C500C520C530C550CAE
:10067000560C580C590C5B0C5C0C5E0C5F0C600C3F
:10068000620C630C650C660C680C690C6B0C6C0CD2
:100690006D0C6F0C700C720C730C740C760C770C68
:1006A000790C7A0C7B0C7D0C7E0C7F0C810C820CFF
:1006B000840C850C860C880C890C8A0C8C0C8D0C97
:1006C0008E0C8F0C910C920C930C950C960C970C35
:1006D000980C9A0C9B0C9C0C9D0C9F0CA00CA10CD4
:1006E000A20CA40CA50CA60CA70CA80CA90CAB0C76
:1006F000AC0CAD0CAE0CAF0CB00CB20CB30CB40C1B
:10070000B50CB60CB70CB80CB90CBA0CBB0CBC0CC5
:10071000BE0CBF0CC00CC10CC20CC30CC40CC50C6D
:10072000C60CC70CC80CC90CCA0CCB0CCB0CCC0C1F
:10073000CD0CCE0CCF0CD00CD10CD20CD30CD40CD5
:10074000D50CD50CD60CD70CD80CD90CDA0CDA0C8D
:10075000DB0CDC0CDD0CDE0CDE0CDF0CE00CE10C49
:10076000E10CE20CE30CE40CE40CE50CE60CE60C0A
:10077000E70CE80CE80CE90CEA0CEA0CEB0CEB0CCF
:10078000EC0CED0CED0CEE0CEE0CEF0CEF0CF00C99
:10079000F10CF10CF20CF20CF30CF30CF30CF40C66
:1007A000F40CF50CF50CF60CF60CF70CF70CF70C3A
:1007B000F80CF80CF80CF90CF90CF90CFA0CFA0C12
:1007C000FA0CFB0CFB0CFB0CFB0CFC0CFC0CFC0CEF
:1007D000FC0CFD0CFD0CFD0CFD0CFD0CFE0CFE0CD0
:1007E000FE0CFE0CFE0CFE0CFE0CFF0CFF0CFF0CB6
:1007F000FF0CFF0CFF0CFF0CFF0CFF0CFF0CFF0CA1
:020800001200E4
:020000040030CA
:0E000000FFFEFEFAFFFEFBFFFFFFFFFFFFFF0C
:00000001FF
